:1008000058EF04F0FF00FF00D9CF6EF0DACF6FF0A1
:10081000AFEF25F0FF00FF00D8CF4DF0E8CF4EF04E
:10082000E0CF4FF0E9CF50F0EACF51F0E1CF52F0F6
:10083000E2CF53F0D9CF54F0DACF55F0F3CF56F0E2
:10084000F4CF57F0F6CF58F0F7CF59F0F8CF5AF071
:10085000F5CF5BF0F238E832010B4C6EF230E83243
:10086000010B4C140009D8B401D001D002D05EECC9
:1008700012F05BC0F5FF5AC0F8FF59C0F7FF58C02F
:10088000F6FF57C0F4FF56C0F3FF55C0DAFF54C05F
:10089000D9FF53C0E2FF52C0E1FF51C0EAFF50C090
:1008A000E9FF4FC0E0FF4EC0E8FF4DC0D8FF100089
:1008B0007DEF25F0E8CF4BF0ECD14B5042EF0EF03E
:1008C0004B5072DA08E15251491805E1515148186C
:1008D00002E150514718D8A41200FF0E186E9D0E69
:1008E000176E74EC08F04B50A3EC1EF08CEF24F064
:1008F0004B505ADA08E15251491805E15151481854
:1009000002E150514718D8A412004B50A3EC1EF03E
:10091000FF0E186E5B0E176E74EC08F04B5054EC23
:100920000BF002E153EF21F04B50A6EF23F04B50B8
:100930003BDA08E15251491805E15151481802E1EA
:10094000505147180BE14B50A3EC1EF0FF0E186EF0
:100950004E0E176E74EC08F00EEF21F04B50D96E6E
:10096000DA6ADF503F0BD8A41200C4C001F0C5C042
:1009700002F0C5EC26F060EC24F00D50E5EC26F01A
:100980000EEF21F04B5010DA08E15251491805E101
:100990005151481802E150514718D8A41200FF0ED7
:1009A000186E7E0E176E74EC08F04B50A3EC1EF020
:1009B0004BC013F0146AFAEF16F04B50F5D908E16A
:1009C0005251491805E15151481802E15051471858
:1009D000D8A41200FF0E186EA70E176E74EC08F064
:1009E0004B50A3EC1EF0086AC80E076E010E096E8C
:1009F0000B6AC80E0A6E4B504DEC0BF0016E026A8A
:100A0000030E046EE80E036E96EC25F001C00CF0A8
:100A100002C00DF0020E46EC1FF04B5094EF1FF099
:100A20004B50C2D908E15251491805E151514818BB
:100A300002E150514718D8A412004B507DEF11F03D
:100A40004B50B2D908E15251491805E151514818AB
:100A500002E150514718D8A41200FF0E186ED90EAB
:100A6000176E74EC08F04B50A3EC1EF04B5039EFAE
:100A700013F04B5099D908E15251491805E15151F1
:100A8000481802E150514718D8A41200FF0E186E02
:100A9000D20E176E74EC08F04B50A3EC1EF04B50C6
:100AA00012EF14F04B5080D908E15251491805E17A
:100AB0005151481802E150514718D8A41200FF0EB6
:100AC000186EED0E176E74EC08F04B50A3EC1EF090
:100AD0004B508FEF15F04B5067D908E15251491830
:100AE00005E15151481802E150514718D8A41200AD
:100AF000FF0E186EF70E176E74EC08F04B50A3EC57
:100B00001EF04B50D6EF14F04B504ED908E1525125
:100B1000491805E15151481802E150514718D8A42D
:100B20001200FF0E186EF20E176E74EC08F04B50A8
:100B3000A3EC1EF04B50FFEF09F04B5035D908E104
:100B40005251491805E15151481802E150514718D6
:100B5000D8A41200FF0E186EE10E176E74EC08F0A8
:100B60004B50A3EC1EF04B50CCEF22F0FF0E186E52
:100B7000230E176E74EC08F04B50A3EC1EF04B5094
:100B8000D96EDA6A0C0ED926DA6ADF50436E4B5002
:100B9000D96EDA6A0B0ED926DA6ADF50446E4B50F2
:100BA000D96EDA6A0A0ED926DA6ADF50456E4B50E2
:100BB000D96EDA6A090ED926DA6ADF50466E4B50D2
:100BC000D96EDA6A080ED926DA6ADF50476E4B50C2
:100BD0003FEC1FF0486E4B50D96EDA6A060ED926EC
:100BE000DA6ADF50496E4B504DEC0BF04924482433
:100BF000472446244524442443245E6E5E50460A1E
:100C0000D8A412004B50D0D808E15251491805E140
:100C10005151481802E150514718D8A41200F29ED1
:100C2000FF0E186E320E176E74EC08F0C7EF20F04E
:100C3000FF0E186EE00E176E74EC08F027D001015D
:100C40004C670BD0086A640E076E096A0B6A0A6E5D
:100C5000000E0D6A0C6A46EC1FF0500E01014C6F3D
:100C6000500CFF0E186E930E176E4B50D96EDA6A49
:100C7000000EDE14196EFC0EDE141A6EFF0EDE146A
:100C80001B6E1F0EDE141C6E74EC08F04B50A3EFAD
:100C90001EF04B50D96EDA6A000EDE14436EFC0E65
:100CA000DE14446EFF0EDE14456E1F0EDE14466E1B
:100CB00046506BE0020A6CE00A0A6EE0120A70E02D
:100CC000D0D74450CEE1435001E1F7D5CAD74450C4
:100CD00019E0040A1BE00C0A1DE0040A1FE01C0ACC
:100CE00021E0040A23E00C0A25E0040A27E02C0A8C
:100CF00029E0040A2BE00C0A2DE0780A2FE0040A10
:100D000031E0AFD7435001E18BD6ABD7435001E17F
:100D1000C9D6A7D7435001E193D6A3D7435001E1E9
:100D2000DAD69FD7435001E1A4D69BD7435001E1C7
:100D300004D797D7435001E17BD793D7435001E1C4
:100D4000E3D68FD7435001E1BBD58BD7435001E1A8
:100D500019D687D7435001E1CBD583D7435001E162
:100D60002CD67FD7435001E1E2D57BD744501C0AF3
:100D700001E077D7435001E162D773D7445001E0D7
:100D800070D7435001E1F2D66CD745509AE069D74D
:100D90004550070A9CE065D74550040AE7E061D753
:100DA0004550070AEBE05DD7D96EDA6ADECF43F033
:100DB000DECF44F0DECF45F0DECF46F03F0E4314E9
:100DC000476E486A496A4A6A010153514A1812003B
:100DD000000E9E6F8A0E9D6F4AD1A451250A04E031
:100DE000A451D7EC26F043D19F6B47D09F8945D0C3
:100DF0009F8F55D09DC0D9FF9EC0DAFFDECFA0F0F7
:100E0000DDCFA1F0020E9D27000E9E23A151A0115F
:100E10001CE1FF0EA16FCB0EA06F17D00001A0C088
:100E2000F6FFA1C0F7FF000EF86E0E0EF76403D0B8
:100E30000800F55005D0F6CFE9FFF7CFEAFFEF50F5
:100E4000D7EC26F00001A04BA12BA0C0F6FFA1C05B
:100E5000F7FF000EF86E0E0EF76403D00800F55091
:100E600005D0F6CFE9FFF7CFEAFFEF50000901E127
:100E7000FED0D4D7C00E9F1312D010D90001A451B8
:100E8000D8B41200640A0BE00D0A09E0050AAEE0CE
:100E90001F0AB0E0060AEEE00D0AAAE0E8D09F5172
:100EA000C00B24E19FA904D09DC0D9FF07D90ED063
:100EB0009DC0D9FF9EC0DAFFDECFA0F0DDCFA1F04C
:100EC000000EA1BFFF0EA26FA36F020E9D27000EA2
:100ED0009E23A3AF62D0030E9F13A31FA21FA11FC7
:100EE000A06D000EA123A223A32357D09FA904D055
:100EF0009DC0D9FFE3D80FD09DC0D9FF9EC0DAFFB7
:100F0000DECF98F0DDCF99F098C0A0F099C0A1F0A5
:100F1000A26BA36B020E9D27000E9E233ED0010EF6
:100F2000A46FA451040D700EF324F66EFD0EF42090
:100F3000F76EF86A000EF8220900F550A05D09006E
:100F4000F550A1590900F550A2590900F550A359CF
:100F50002BE3A42BA4510A0A27E0E3D7010EA46FC8
:100F6000A451040D980EF324F66EFD0EF420F76ED6
:100F7000F86A000EF8220900F550A05D0900F5504E
:100F8000A1590900F550A2590900F550A3590CE3E5
:100F9000A42BA451080A08E0E3D79F51C00BBFE07F
:100FA000800ADCE0400ABBE09F51030B03E02D0EFA
:100FB000D7EC26F00001A4519B6F9C6B9BBF9C0754
:100FC0004ED087D8700E9825F66EFD0E55D8A0C06D
:100FD00072F0A1C073F0A2C074F0A3C075F091ECE0
:100FE00022F075C082F074C081F073C080F072C0CE
:100FF0007FF00A0E836F000E846B856B866B75EC39
:1010000023F07F51300FA46F27D0A0C072F0A1C091
:1010100073F0A2C074F0A3C075F05BD8980E982549
:10102000F66EFD0E29D891EC22F072510F0B9A6FDB
:10103000DF0E9A25F66EF76AFE0EF722F86A000EAA
:10104000F8220800F5CFA4F007D09F51C00BB9E0FB
:10105000800ADBE0400AB5E0A451D7EC26F000019D
:101060009B07D8A09C079B29D8B49C29EEE10001DE
:1010700015D8A467B2D612009921F76EF86A000E4F
:10108000F8220900F5CF76F00900F5CF77F00900D6
:10109000F5CF78F00A00F5CF79F012008851986FFB
:1010A0008951996F884B892B98C0F6FF99C0F7FF3B
:1010B000000EF86E0800F5CFA4F012009EC0DAFF13
:1010C000DECFA0F0DECFA1F0DECFA2F0DECFA3F026
:1010D000040C9BC098F09CC099F0D8909837993731
:1010E000D890983799371200190E2C6E000E2D6E7D
:1010F0000F0E2D6E5F0E2C642D6A45D13350250ADC
:1011000004E03350ECEC26F03ED12E6A45D02E8818
:1011100043D02E8E52D02CC0D9FF2DC0DAFFDECFA7
:101120002FF0DDCF30F0020E2C26000E2D22305095
:101130002F101AE1FF0E306ECB0E2F6E15D02FC080
:10114000F6FF30C0F7FF000EF86E0E0EF76403D006
:101150000800F55005D0F6CFE9FFF7CFEAFFEF50D2
:10116000ECEC26F02F4A302A2FC0F6FF30C0F7FFF4
:10117000000EF86E0E0EF76403D00800F55005D08F
:10118000F6CFE9FFF7CFEAFFEF50000901E1FBD00E
:10119000D6D7C00E2E1211D00CD93350D8B41200AD
:1011A000640A0BE00D0A09E0050AB1E01F0AB3E08A
:1011B000060AEFE00D0AADE0E6D02E50C00B24E1A8
:1011C0002EA804D02CC0D9FF04D90ED02CC0D9FF32
:1011D0002DC0DAFFDECF2FF0DDCF30F0000E30BEB5
:1011E000FF0E316E326E020E2C26000E2D2232AE14
:1011F00062D0030E2E12321E311E301E2F6C000ED6
:1012000030223122322257D02EA804D02CC0D9FF50
:10121000E0D80FD02CC0D9FF2DC0DAFFDECF27F0E9
:10122000DDCF28F027C02FF028C030F0316A326AB5
:10123000020E2C26000E2D223ED0010E336E3350AE
:10124000040D700EF324F66EFD0EF420F76EF86AAE
:10125000000EF8220900F5502F5C0900F5503058B7
:101260000900F55031580900F55032582BE3332A64
:1012700033500A0A27E0E3D7010E336E3350040DD2
:10128000980EF324F66EFD0EF420F76EF86A000E49
:10129000F8220900F5502F5C0900F550305809007C
:1012A000F55031580900F55032580CE3332A3350C9
:1012B000080A08E0E3D72E50C00BBFE0800ADCE04C
:1012C000400ABBE02E50030B03E02D0EECEC26F0A1
:1012D00033502A6E2B6A2ABE2B064ED085D8700E4C
:1012E0002724F66EFD0E53D82FC001F030C002F057
:1012F00031C003F032C004F007EC23F004C011F059
:1013000003C010F002C00FF001C00EF00A0E126E02
:10131000000E136A146A156AD7EC23F00E50300FD2
:10132000336E27D02FC001F030C002F031C003F07F
:1013300032C004F059D8980E2724F66EFD0E27D837
:1013400007EC23F001500F0B296EDF0E2924F66EF7
:10135000F76AFE0EF722F86A000EF8220800F5CFB1
:1013600033F007D02E50C00BB9E0800ADBE0400A12
:10137000B5E03350ECEC26F02A06D8A02B062A283C
:10138000D8B42B28EFE115D83366B8D61200282040
:10139000F76EF86A000EF8220900F5CF05F0090093
:1013A000F5CF06F00900F5CF07F00A00F5CF08F0F9
:1013B00012001750276E1850286E174A182A27C097
:1013C000F6FF28C0F7FF000EF86E0800F5CF33F0E7
:1013D00012002DC0DAFFDECF2FF0DECF30F0DECFEF
:1013E00031F0DECF32F0040C2AC027F02BC028F0F9
:1013F000D89027362836D890273628361200E8CFDE
:101400003EF03E50D96EDA6AC00EDE14386EFF0E22
:10141000DE14396EFF0EDE143A6EFF0EDE143B6EE4
:101420000DD13E5041D911E03E5037D90101036F33
:10143000026A060E016E03C103F060EC25F007ECB2
:1014400027F03E5094EC1FF007D03E503BD903C12B
:10145000CDF031D975EC10F0FE0E186E2E0EEBD0DB
:101460003E5022D911E03E5018D903E00101028B11
:1014700002D00101029B34D960EC25F007EC27F083
:101480003E5094EC1FF00CD03E501CD901010239A3
:10149000E842070B010B0001CD6F0DD975EC10F080
:1014A000FD0E186EFD0EC7D03E50FED811E03E5026
:1014B000F4D803E00101028502D00101029510D9A0
:1014C00060EC25F007EC27F03E5094EC1FF00CD0B8
:1014D0003E50F8D801010241E8423F0B010B0001E8
:1014E000CD6FE9D875EC10F0FE0E186E160EA3D075
:1014F0003E50DAD811E03E50D0D803E00101028717
:1015000002D001010297ECD860EC25F007EC27F03F
:101510003E5094EC1FF00CD03E50D4D8010102395B
:10152000E8461F0B010B0001CD6FC5D875EC10F01C
:10153000FE0E186E730E7FD03E50B6D811E03E50AE
:10154000ACD803E00101028902D001010299C8D898
:1015500060EC25F007EC27F03E5094EC1FF00BD028
:101560003E50B0D8010102390F0B010B0001CD6FC5
:10157000A2D875EC10F0FE0E186E450E5CD03E50F1
:10158000D96EDA6A040ED926DA6A010EDF641FD03A
:101590003E50D96EDA6A060ED926DA6ADF50356E09
:1015A000346A3E507AD834243C6E000E35203D6EAD
:1015B0003D50800A800F010ED8B43C5C04E33CC06F
:1015C00007F13DC008F13E5094EC1FF00DD03E50A5
:1015D000D96EC9EC14F007C1CDF00101085100012A
:1015E000CE6F69D875EC10F0FE0E186E890E23D000
:1015F0003E505AD811E03E5050D803E00101028D10
:1016000002D00101029D6CD860EC25F007EC27F0B8
:101610003E5094EC1FF00CD03E5054D801010245CE
:10162000E846030B010B0001CD6F45D875EC10F0B7
:10163000FE0E186EB50E176E74EF08F038C034F059
:1016400039C035F03AC036F03BC037F03750020AA7
:10165000D8A412001DD035501C0A04E0010AD8A4F9
:10166000120009D03450C4E0800A01E1DAD6400A01
:10167000D8A41200F5D6345001E116D7400A01E192
:1016800037D7C00A01E158D7400AD8A4120077D74B
:101690003650070AD8A41200DED7D96EDA6A050ED2
:1016A000D926DA6ADF501200D96EDA6A040ED9261A
:1016B000DA6ADF501200000E116EC80E106E010EB5
:1016C000126E010CD96EDA6A0001DECFC8F0DECFEF
:1016D000C9F0DECFCAF0DECFCBF0010ECC6F010C2B
:1016E000026A040E016E0251FC0B036E12000F0120
:1016F00020B735D00F0E0001736F210EFDD884EC9A
:101700001BF020EE04F0F1D8256F000120EE05F06B
:10171000ECD8266F000120EE06F0E7D8276F000115
:1017200020EE07F0E2D8286F000120EE08F0DDD8A7
:10173000296F000120EE09F0D8D82A6F000120EEB1
:101740000AF0D3D82B6F000120EE0BF0CED82C6F0F
:10175000000120EE0CF0C9D82D6F2087120010B7C1
:1017600035D00F0E0001736F110EC6D884EC1BF03C
:1017700020EE04F0BAD8156F000120EE05F0B5D8C0
:10178000166F000120EE06F0B0D8176F000120EEB2
:1017900007F0ABD8186F000120EE08F0A6D8196F3B
:1017A000000120EE09F0A1D81A6F000120EE0AF026
:1017B0009CD81B6F000120EE0BF097D81C6F000126
:1017C00020EE0CF092D81D6F1087120000B735D0B4
:1017D0000F0E0001736F010E8FD884EC1BF020EE0A
:1017E00004F083D8056F000120EE05F07ED8066F67
:1017F000000120EE06F079D8076F000120EE07F017
:1018000074D8086F000120EE08F06FD8096F00014E
:1018100020EE09F06AD80A6F000120EE0AF065D8C0
:101820000B6F000120EE0BF060D80C6F000120EE72
:101830000CF05BD80D6F008712000E01B0B71BD003
:101840000E0E0001736FB10E57D884EC1BF0B4D8A4
:10185000B56F62D8B66F6AD8B76F72D8B86FA2D8B2
:10186000B96F82D8BA6F8AD8BB6F92D8BC6F72D862
:10187000BD6FB0871200C0B71BD00E0E0001736F92
:10188000C10E3AD884EC1BF097D8C56F45D8C66F07
:101890004DD8C76F55D8C86F85D8C96F65D8CA6F7E
:1018A0006DD8CB6F75D8CC6F55D8CD6FC08712006F
:1018B000D0B712000E0E0001736FD10E1DD884EC4C
:1018C0001BF07AD8D56F28D8D66F30D8D76F38D8D4
:1018D000D86F68D8D96F48D8DA6F50D8DB6F58D82E
:1018E000DC6F38D8DD6FD08712008151D926825144
:1018F000DA22DF500F011200726F81C0D9FF82C05F
:10190000DAFFDECF74F0DECF75F0DECF76F0DECF1B
:1019100077F083C078F01200000120EE05F08151CD
:10192000D9268251DA22DF500E011200000120EE8A
:1019300006F08151D9268251DA22DF500E011200C1
:10194000000120EE07F08151D9268251DA22DF50C2
:101950000E011200000120EE0CF08151D9268251B7
:10196000DA22DF500E011200000120EE09F0815151
:10197000D9268251DA22DF500E011200000120EE3A
:101980000AF08151D9268251DA22DF500E0112006D
:10199000000120EE0BF08151D9268251DA22DF506E
:1019A0000E011200000120EE08F08151D92682516B
:1019B000DA22DF500E01120020EE04F08151D92608
:1019C0008251DA22DF500E011200EAD00F0E616F51
:1019D000610E606FB3510D0D000EF3240001626FB4
:1019E000020EF420636F010E646F0DEC1BF0B35117
:1019F00019D965CFDFFFF0D866CFDFFFB3510AD921
:101A000067CFDFFFB351FED868CFDFFFB3511AD9DC
:101A100069CFDFFFB3510ED96ACFDFFFB35122D9AF
:101A20006BCFDFFFB35116D96CCFDFFFB35122D993
:101A30006DCFDFFF609EC8D00F0E0001616F310EC9
:101A4000D5D80DEC1BF0B351EDD835CFDFFFC4D89E
:101A500036CFDFFFB351DED837CFDFFFB351D2D857
:101A600038CFDFFFB351EED839CFDFFFB351E2D823
:101A70003ACFDFFFB351F6D83BCFDFFFB351EAD8FF
:101A80003CCFDFFFB351F6D80F013DCFDFFF309FD2
:101A90009BD00E0E0001616F810EA8D80DEC1BF0DB
:101AA000B351C0D885CEDFFF97D886CEDFFFB351C4
:101AB000B1D887CEDFFFB351A5D888CEDFFFB351B1
:101AC000C1D889CEDFFFB351B5D88ACEDFFFB3517D
:101AD000C9D88BCEDFFFB351BDD88CCEDFFFB35159
:101AE000C9D80E018DCEDFFF809F6ED00E0E000193
:101AF000616F910E7BD80DEC1BF0B35193D895CE4E
:101B0000DFFF6AD896CEDFFFB35184D897CEDFFFD0
:101B1000B35178D898CEDFFFB35194D899CEDFFF78
:101B2000B35188D89ACEDFFFB3519CD89BCEDFFF4C
:101B3000B35190D89CCEDFFFB3519CD80E019DCEFF
:101B4000DFFF909F41D00E0E0001616FA10E4ED8B5
:101B50000DEC1BF0B35166D8A5CEDFFF3DD8A6CE65
:101B6000DFFFB35157D8A7CEDFFFB3514BD8A8CE74
:101B7000DFFFB35167D8A9CEDFFFB3515BD8AACE40
:101B8000DFFFB3516FD8ABCEDFFFB35163D8ACCE1C
:101B9000DFFFB3516FD80E01ADCEDFFFA09F14D091
:101BA0006F500F0B00016C6F6D6B6D510DE16C513F
:101BB00001E10CD7010A01E13FD7030A01E169D72E
:101BC000010A94E0070ABFE00001B32B0F0EB31720
:101BD0005D2A5D1677920F0C0001B3510D0D050EB5
:101BE000F324D96E020EF420DA6E1200606FB35146
:101BF0000D0D000EF324626F020EF420636F010ED0
:101C0000646F010C0D0D070EF324D96E020EF42043
:101C1000DA6E12000D0D060EF324D96E020EF420BA
:101C2000DA6E12000D0D040EF324D96E020EF420AC
:101C3000DA6E12000D0D090EF324D96E020EF42097
:101C4000DA6E12000D0D080EF324D96E020EF42088
:101C5000DA6E12000D0D0B0EF324D96E020EF42075
:101C6000DA6E12000D0D0A0EF324D96E020EF42066
:101C7000DA6E12000D0D0C0EF324D96E020EF42054
:101C8000DA6E1200E8CF42F0CFD0FF0E186EBA0E17
:101C9000176E74EC08F04250A3EC1EF0040E010124
:101CA000006F096B0A6B0D6B0E6B000E086A076AFA
:101CB000A7EC17F00AEF27F0FF0E186E730E176EE1
:101CC00074EC08F04250A3EC1EF00101096B0A6BA2
:101CD000010E006FF9EF26F0FF0E186EC30E176E9F
:101CE00074EC08F04250A3EC1EF00101006B096B8C
:101CF0000A6B0D6B0E6B086A076AA7EF17F0230ECD
:101D000001014D6F230CFF0E186E890E176E74ECD7
:101D100008F087D0FE0E186E9F0E176E74EC08F058
:101D20004250A3EC1EF04250D96EDA6A0C0ED9264E
:101D3000DA6ADF503A6E4250D96EDA6A0B0ED92653
:101D4000DA6ADF503B6E4250D96EDA6A0A0ED92643
:101D5000DA6ADF503C6E4250D96EDA6A090ED92633
:101D6000DA6ADF503D6E4250D96EDA6A080ED92623
:101D7000DA6ADF503E6E42503FEC1FF03F6E425039
:101D8000D96EDA6A060ED926DA6ADF50406E425002
:101D90004DEC0BF040243F243E243D243C243B24C6
:101DA0003A245E6E5E50460AD8A412004250D96EA4
:101DB000DA6ADECF3AF0DECF3BF0DECF3CF0DECFAA
:101DC0003DF03F0E3A143E6E3F6A406A416A01019F
:101DD0005351411808E15251401805E151513F1843
:101DE00002E150513E18D8A41200F29EFF0E186E68
:101DF000320E176E74EC08F0C7EF20F0FF0E186E6D
:101E0000E70E176E74EC08F00CD0FF0E186EFC0E87
:101E1000176E74EF08F0FF0E186EB10E176E74ECAB
:101E200008F04250A3EF1EF04250D96EDA6AC00E9D
:101E3000DE143A6EFF0EDE143B6EFF0EDE143C6EB7
:101E4000FF0EDE143D6E3D5033E0080A34E0120A06
:101E500036E0E1D73B5005E0010A10E0030A12E04A
:101E6000DAD73A5001E111D7400A01E135D7C00A6B
:101E7000D8B41200400A01E146D7CDD73A50800AC3
:101E8000BDE0C9D73A50400A01E139D7C00A01E1A3
:101E900013D7C1D73B501C0ABEE13A50B6E0BBD7BE
:101EA0003B50010AB8E13A50800A01E133D7B3D779
:101EB0003C50D0E0B0D73C50040AECE0ACD73C50EA
:101EC000070AEEE0A8D70101000501E0ECD0D8EC4C
:101ED00021F029500101175D316E2A501859326ED8
:101EE00031C027F132C028F1000E28BFFF0E296F44
:101EF0002A6F21EE3BF0E0D8DAEC24F004C032F196
:101F000003C031F102C030F101C02FF1010121EE17
:101F10003DF0D2D8DAEC24F0010133510124336FC3
:101F200034510220346F35510320356F365104206F
:101F3000366F3651800A800F08E1000E355D05E1ED
:101F4000750E345D02E1310E335D06E3300E336F02
:101F5000750E346F356B366B3651800A810F08E190
:101F6000FF0E355D05E18A0E345D02E1D00E335D72
:101F700006E2D00E336F8A0E346F35693669275109
:101F80002B5D016E28512C59026E29512D59036E7B
:101F90002A512E59046E21EE3FF0DECF05F0DDCF41
:101FA00006F0000E06BEFF0E076E086EDAEC24F097
:101FB00004C03AF103C039F102C038F101C037F171
:101FC00027C12BF128C12CF129C12DF12AC12EF1F5
:101FD000010133512F25316E34513021326E35518C
:101FE0003121336E36513221346E375131240B6E2C
:101FF000385132200C6E395133200D6E3A51342055
:102000000E6E00EC25F00EC044F10DC043F10CC083
:1020100042F10BC041F1016AC00E026E7F0E036EE9
:10202000440E046E41C105F042C106F043C107F001
:1020300044C108F0B4EC24F003E250D8440E446FDD
:1020400041C101F042C102F043C103F044C104F0B8
:10205000056AC00E066E7F0E076EC40E086EB4ECE5
:1020600024F003E23BD8C40E446F41C10BF042C1DF
:102070000CF043C10DF044C10EF0E2EC1FF00BC0B8
:102080000DF10CC00EF17DEC20F001C007F002C094
:1020900008F0A7EC17F07DEC20F001C00FF002C0B3
:1020A00010F048EF1EF0000E086A076AA7EC17F060
:1020B000106A0F6A48EF1EF0DECF01F0DDCF02F0AC
:1020C000000E02BEFF0E036E046E27C105F028C18C
:1020D00006F029C107F02AC108F012000101416B86
:1020E000C00E426F7F0E436F7F0C0F0120B71BD0D5
:1020F0000F0E026E210EA9D8F1EC1BF0E6D80F01ED
:10210000256FDBD8266FE9D8276FEFD8286FCDD899
:10211000296FB3D82A6FB9D82B6FBFD82C6FA5D829
:102120002D6F2087120010B71BD00F0E026E110EFC
:102130008CD8F1EC1BF0C9D80F01156FBED8166F03
:10214000CCD8176FD2D8186FB0D8196F96D81A6F2D
:102150009CD81B6FA2D81C6F88D81D6F10871200E7
:1021600000B71BD00F0E026E010E6FD8F1EC1BF002
:10217000ACD80F01056FA1D8066FAFD8076FB5D8DF
:10218000086F93D8096F79D80A6F7FD80B6F85D8FD
:102190000C6F6BD80D6F008712000E01B0B71BD00B
:1021A0000E0E026EB10E51D8F1EC1BF08ED80E015E
:1021B000B56F83D8B66F91D8B76F97D8B86F75D809
:1021C000B96F5BD8BA6F61D8BB6F67D8BC6F4DD899
:1021D000BD6FB0871200C0B71BD00E0E026EC10ECD
:1021E00034D8F1EC1BF071D80E01C56F66D8C66FFC
:1021F00074D8C76F7AD8C86F58D8C96F3ED8CA6F1D
:1022000044D8CB6F4AD8CC6F30D8CD6FC08712007E
:10221000D0B712000E0E026ED10E17D8F1EC1BF0E3
:1022200054D80E01D56F49D8D66F57D8D76F5DD81F
:10223000D86F3BD8D96F21D8DA6F27D8DB6F2DD86C
:10224000DC6F13D8DD6FD0871200016E10C0D9FF8C
:1022500011C0DAFFDECF03F0DECF04F0DECF05F0F1
:10226000DECF06F012C007F0120020EE0CF0105086
:10227000D9261150DA22DF50120020EE09F010505A
:10228000D9261150DA22DF50120020EE0AF0105049
:10229000D9261150DA22DF50120020EE0BF0105038
:1022A000D9261150DA22DF50120020EE08F010502B
:1022B000D9261150DA22DF50120020EE05F010501E
:1022C000D9261150DA22DF50120020EE04F010500F
:1022D000D9261150DA22DF50120020EE06F01050FD
:1022E000D9261150DA22DF50120020EE07F01050EC
:1022F000D9261150DA22DF501200E8CF1BF01B5014
:10230000D96EDA6AC00EDE14176EFF0EDE14186E78
:10231000FF0EDE14196EFF0EDE141A6EA1D0010E30
:10232000016F010C015118E01B50F7EC1EF0136E09
:102330000051040A010ED8B4000E131402E0010E7D
:10234000006F016B026A030E016E0151FC0B036EFC
:1023500060EC25F007EC27F01B5054EC0BF00EE17D
:102360001B50D96EC9EC14F009C1CDF001010A511E
:102370000001CE6F5BEC0BF075EF10F01B50D96EC7
:10238000DA6A040ED926DA6A010EDF64010C010153
:102390000051040A25E01B50F7EC1EF0000924E070
:1023A0004F51800A750F04E24F2B0AEC27F01CD026
:1023B0001B50D96EDA6A060ED926DA6ADF50146E1F
:1023C000136A1B504DEC0BF01324096F000E142000
:1023D0000A6F010E006FF9EC26F0280E4E6F04D044
:1023E000096B0A6B0D6B0E6B010121EE09F0DE52D9
:1023F000DD50800A7C0F000ED8B4DF5C04E3030ECE
:102400000A6F0969FF0C21EE09F0DE52DD50800AE7
:10241000840F010ED8B4DF5CD8B01200FC0E0A6F36
:10242000010E096F010C1B5054EC0BF007E11B501F
:10243000D96EC9EC14F047C1CDF09CD71B5054ECB9
:102440000BF0D8B412001B504DEC0BF0476F026A32
:10245000050E016E47C103F060EC25F007EF27F091
:1024600017C013F018C014F019C015F01AC016F0F8
:102470001650020AD8A412001CD0145006E0010A1B
:1024800011E0030AD8A4120012D0135001E14AD778
:10249000400A01E144D7C00A01E144D7400AD8A468
:1024A0001200C1D71350400AD8A412003BD71350D2
:1024B000FBD71550070AD8A41200DFD7E00ED76E5D
:1024C000CF0ED66E0001C42B000EC523C623C72332
:1024D000F29490EC1AF064EC26F00001C4B136D00E
:1024E00001014C0506E1086A640EBCD8030E46ECF7
:1024F0001FF001014C51D8A44C074C6703D0006B6E
:102500000AEC27F001014D0506E1086A320EAAD84F
:10251000010E46EC1FF001014D51D8A44D074D6747
:1025200003D0006B0AEC27F001014E51D8A44E07EE
:102530004E050CE14F6B096B0A6B0D6B0E6B0AECD1
:1025400027F0000E086A076AA7EC17F0C4C00EF067
:10255000C5C00FF0C6C010F0C7C011F0050E126E56
:10256000000E136A146A156AD7EC23F011500E108E
:102570000F1010100EE1DEEC26F02BC013F12CC072
:1025800014F1D8EC21F029C019F12AC01AF198EC05
:1025900021F0C4C00EF0C5C00FF0C6C010F0C7C017
:1025A00011F00A0E126E000E136A146A156AD7EC47
:1025B00023F011500E100F101010D8B47DEC20F045
:1025C000C4C00EF0C5C00FF0C6C010F0C7C011F0F7
:1025D000140E126E000E136A146A156AD7EC23F0FB
:1025E00011500E100F10101012E101014C6707D0AE
:1025F000096B0A6B000E086A076AA7EC17F04667BA
:1026000005D05EEC1CF045C146F101D04607C4C0C0
:102610000EF0C5C00FF0C6C010F0C7C011F0640EB8
:10262000126E000E136A146A156AD7EC23F011506B
:102630000E100F10101006E134EC24F029C005F143
:102640002AC006F1C4C00EF0C5C00FF0C6C010F01D
:10265000C7C011F0E80E126E030E136E146A156AED
:10266000D7EF23F0076E096A0B6A0A6E0D6A0C6ACF
:102670001200E8CF1BF01B50D96EDA6AC00EDE14D0
:10268000176EFF0EDE14186EFF0EDE14196EFF0EAD
:10269000DE141A6E97D001010151080AD8B4120055
:1026A0000051040A02E0080E016F026A030E016E77
:1026B0000151FC0B036E60EC25F007EC27F0030ED4
:1026C00001013C6FE80E3B6F3E6B640E3D6F406B4B
:1026D0003F6F336B346B356B366B1200090E0101A3
:1026E000016F090C1B5054EC0BF00EE11B50D96E1E
:1026F000C9EC14F015C1CDF0010116510001CE6FE7
:102700005BEC0BF075EF10F01B50D96EDA6A040E1B
:10271000D926DA6A010EDF64010C01010051040AB6
:1027200012E01B50D96EDA6A060ED926DA6ADF503B
:10273000146E136A1B504DEC0BF01324156F000E32
:102740001420166F02D0156B166B21EE15F0DE52B9
:10275000DD50800A460F990ED8B4DF5C05E33A0ECF
:10276000166F980E156F980C21EE15F0DE52DD50A5
:10277000800ABB0F680ED8B4DF5CD8B01200C50E5B
:10278000166F680E156F680C1B5054EC0BF007E1C8
:102790001B50D96EC9EC14F047C1CDF0B1D71B5016
:1027A00054EC0BF0D8B412001B504DEC0BF00101AF
:1027B000476F026A050E016E47C103F060EC25F019
:1027C00007EF27F017C013F018C014F019C015F068
:1027D0001AC016F01650020AD8A412001ED01450C7
:1027E000080A06E0010A11E0030AD8A4120012D078
:1027F000135001E150D7400A01E170D7C00A01E14E
:1028000071D7400AD8A41200BFD71350800AD8A4A9
:10281000120068D71350400AFAD71550070AD8A4F7
:102820001200DDD7E8CF1BF01B50D96EDA6AC00E5C
:10283000DE14176EFF0EDE14186EFF0EDE14196E16
:10284000FF0EDE141A6E75D001010151080AD8B4CA
:1028500012000051040AD8B41200080E016F080CCF
:10286000090E0101016F090C1B5054EC0BF00DE136
:102870001B50D96E8ED815C1CDF001011651000143
:10288000CE6F5BEC0BF075EF10F01B50D96EDA6A6F
:10289000040ED926DA6A010EDF64010C0101005131
:1028A000040A12E01B50D96EDA6A060ED926DA6ADB
:1028B000DF50146E136A1B504DEC0BF01324156F90
:1028C000000E1420166F02D0156B166B21EE15F05A
:1028D000DE52DD50800A7C0F010ED8B4DF5C04E3C9
:1028E000030E166F1569FF0C21EE15F0DE52DD5058
:1028F000800A840F010ED8B4DF5CD8B01200FC0E41
:10290000166F010E156F010C1B5054EC0BF006E115
:102910001B50D96E3ED847C1CDF0B3D71B5054ECF5
:102920000BF0D8B412001B504DEC0BF00101476FB7
:10293000120017C013F018C014F019C015F01AC017
:1029400016F01650020AD8A412001ED01450080A1D
:1029500006E0010A11E0030AD8A4120012D01350B5
:1029600001E172D7400A01E17BD7C00A01E17CD7BF
:10297000400AD8A41200C8D71350800AD8A4120065
:1029800073D71350400AFAD71550070AD8A412007B
:10299000DDD7DA6A0001DECFC8F0DECFC9F0DECFC6
:1029A000CAF0DECFCBF0020ECC6F020CE8CF1BF0EA
:1029B0001B50D96EDA6AC00EDE14176EFF0EDE14DD
:1029C000186EFF0EDE14196EFF0EDE141A6E77D02D
:1029D00001010151080AD8B412000051040AD8B408
:1029E0001200080E016F080C090E0101016F090C9D
:1029F0001B5054EC0BF00EE11B50D96EC9EC14F0D7
:102A000015C1CDF0010116510001CE6F5BEC0BF04A
:102A100075EF10F01B50D96EDA6A040ED926DA6A07
:102A2000010EDF64010C01010051040A12E01B5089
:102A3000D96EDA6A060ED926DA6ADF50146E136A86
:102A40001B504DEC0BF01324156F000E1420166F65
:102A500002D0156B166B21EE15F0DE52DD50800AA8
:102A60007C0F010ED8B4DF5C04E3030E166F15690A
:102A7000FF0C21EE15F0DE52DD50800A840F010EAE
:102A8000D8B4DF5CD8B01200FC0E166F010E156FC3
:102A9000010C1B5054EC0BF007E11B50D96EC9EC34
:102AA00014F047C1CDF0B2D71B5054EC0BF0D8B4A2
:102AB00012001B504DEC0BF00101476F120017C0C4
:102AC00013F018C014F019C015F01AC016F0165003
:102AD000020AD8A412001ED01450080A06E0010A07
:102AE00011E0030AD8A4120012D0135001E170D7EC
:102AF000400A01E179D7C00A01E17AD7400AD8A497
:102B00001200C7D71350800AD8A4120071D71350EF
:102B1000400AFAD71550070AD8A41200DDD7E8CF2B
:102B20001BF01B50D96EDA6AC00EDE14176EFF0E52
:102B3000DE14186EFF0EDE14196EFF0EDE141A6E10
:102B400077D001010151080AD8B412000051040ADB
:102B5000D8B41200080E016F080C090E0101016FB4
:102B6000090C1B5054EC0BF00EE11B50D96EC9EC54
:102B700014F015C1CDF0010116510001CE6F5BECD0
:102B80000BF075EF10F01B50D96EDA6A040ED926DF
:102B9000DA6A010EDF64010C01010051040A12E03F
:102BA0001B50D96EDA6A060ED926DA6ADF50146E27
:102BB000136A1B504DEC0BF01324156F000E1420FC
:102BC000166F02D0156B166B21EE15F0DE52DD503C
:102BD000800A7C0F010ED8B4DF5C04E3030E166F8D
:102BE0001569FF0C21EE15F0DE52DD50800A840FCE
:102BF000010ED8B4DF5CD8B01200FC0E166F010EC7
:102C0000156F010C1B5054EC0BF007E11B50D96EF3
:102C1000C9EC14F047C1CDF0B2D71B5054EC0BF007
:102C2000D8B412001B504DEC0BF00101476F12009D
:102C300017C013F018C014F019C015F01AC016F020
:102C40001650020AD8A412001ED01450080A06E03A
:102C5000010A11E0030AD8A4120012D0135001E1B6
:102C600070D7400A01E179D7C00A01E17AD7400A5A
:102C7000D8A41200C7D71350800AD8A4120071D765
:102C80001350400AFAD71550070AD8A41200DDD70E
:102C9000BBAE08D0BCCF79F0A5D8BBB87981BBBAA0
:102CA00079830BD0BCCF79F09DD8BBB87981BBBA02
:102CB0007983796D7A1FD8B07A2B010102AD05D0E6
:102CC0000001796D7A1FD8B07A2B00017751761107
:102CD00047E07651795D726F77517A59736FEFECF7
:102CE00025F07351800A800F150ED8B4725D1BE376
:102CF0007751800A786F7951765D7A51800A7859D8
:102D000004E3140E7927000E0CD07A51800A786FF4
:102D10007651795D7751800A785909E3EC0E79276D
:102D2000FF0E7A2304D076C079F077C07AF07A511A
:102D3000800A7D0FFF0ED8B4795D03E3030E7A6F2E
:102D400079697A51800A840F020ED8B4795D04E261
:102D5000FC0E7A6F010E796F79C076F07AC077F049
:102D6000010102AD05D00001766D771FD8B0772B39
:102D7000000177AF0AD0766D771FD8B0772BBB9E56
:102D8000BB84BB860A0E8A120ED07751800A800F50
:102D9000010ED8B4765D02E3BB8EF2D7010102AB1F
:102DA00002D0BB94BB9676C078F0010E0001781774
:102DB000783BBB507819EF0B7819BB6E77357733BA
:102DC000763376C078F0010E7817783B7847BB50A1
:102DD0007819DF0B7819BB6E77357733763376C089
:102DE000BCFF12007A6BD89079377A37D890793750
:102DF0007A371200A4D8156E15C016F0176A186A33
:102E0000196A01015351191808E15251181805E1C6
:102E10005151171802E150511618D8A4120020EE93
:102E20000CF01350D9261450DA22DF50156E20EE24
:102E30000BF01350D9261450DA22DF50166E20EE14
:102E40000AF01350D9261450DA22DF50176E20EE04
:102E500009F01350D9261450DA22DF50186E20EEF4
:102E600008F01350D9261450DA22DF50196E20EEE4
:102E700007F01350D9261450DA22DF501A6E20EED4
:102E800006F01350D9261450DA22DF501B6E57D8A3
:102E90001B241A24192418241724162415241D6E03
:102EA0001D50460AD8A4120020EE06F01350D92671
:102EB0001450DA22DF50506F516B526B536B13C0BA
:102EC000D9FF14C0DAFFC00EDE14156EFF0EDE143B
:102ED000166EFF0EDE14176EFF0EDE14186E5051C4
:102EE0001510196E515116101A6E525117101B6E93
:102EF000535118101C6E13C0D9FF14C0DAFF19C04B
:102F0000DEFF1AC0DEFF1BC0DEFF1CC0DDFFD906DE
:102F1000D906026A020E016E50C103F060EC25F082
:102F200007EC27F0130E106E000E116E0F0E116ECF
:102F30005F0E1064116A010E126E75EF10F020EE34
:102F400005F01350D9261450DA22DF501200BBAE20
:102F500008D0BCCF0AF09ED8BBB80A80BBBA0A82A0
:102F60000BD0BCCF0AF096D8BBB80A80BBBA0A8295
:102F70000A6C0B1ED8B00B2A010102AD04D00A6CFA
:102F80000B1ED8B00B2A0850071047E007500A5C08
:102F9000016E08500B58026E03EC26F00250800AB6
:102FA000800F150ED8B4015C1BE30850800A096E2F
:102FB0000A50075C0B50800A095804E3140E0A26D5
:102FC000000E0CD00B50800A096E07500A5C0850A6
:102FD000800A095809E3EC0E0A26FF0E0B2204D0E2
:102FE00007C00AF008C00BF00B50800A7D0FFF0EDF
:102FF000D8B40A5C03E3030E0B6E0A680B50800A18
:10300000840F020ED8B40A5C04E2FC0E0B6E010EB3
:103010000A6E0AC007F00BC008F002AD04D0076CBE
:10302000081ED8B0082A08AE0AD0076C081ED8B00F
:10303000082ABB9EBB84BB860A0E8A120DD008509C
:10304000800A800F010ED8B4075C02E3BB8EF2D772
:1030500002AB02D0BB94BB9607C009F0010E091663
:10306000093ABB500918EF0B0918BB6E0834083237
:10307000073207C009F0010E0916093A0946BB508C
:103080000918DF0B0918BB6E08340832073207C075
:10309000BCFF12000B6AD8900A360B36D8900A365D
:1030A0000B361200500E01014C6F096B0A6B0D6B51
:1030B0000E6B010E456F45C146F1700ED3129B8C0D
:1030C0004E6B42EC23F0000E0001776B766B48EC00
:1030D00016F001014C6B0001736B640E726F746B20
:1030E000766B756F000E786B776B30EC20F0000E0E
:1030F000776B766B48EC16F0736B020E726F40ECD8
:1031000026F0F3EC26F00101506F516B526B536BBC
:103110000001736B030E726F40EC26F00101016F2A
:103120000001736B040E726F40EC26F00101026F18
:103130000001736B050E726F40EC26F00101476FC2
:103140000001736B060E726F40EC26F00101036FF5
:10315000FE0E0001896FCA0E886FE8EC06F0FD0EC6
:10316000896FB80E886FFF0E8B6F670E8A6F8D6B3D
:10317000010E8C6F8F6B050E8E6F34EC26F072C0D3
:1031800090F073C091F0936B926B030E736FFD0E12
:10319000726F40EC26F00001946F956B030E736F15
:1031A000FE0E726F40EC26F00001966F976BE8EC14
:1031B00006F0FF0E896F010E886F0001F0CE8AF0D5
:1031C0008B6BF1CE8CF08D6BF2CE8EF08F6BF3CEDD
:1031D00090F0916BE8EC06F0FFD7E8CF89F0800E15
:1031E0006F6E6E38E832070B040AF9E1100E0E011B
:1031F000716F716F320E726F540E736F760E746F43
:10320000980E756FBA0E766FDC0E776FFE0E786FC4
:103210003F0E0001816F826B83691F0E846F010E68
:10322000856F000E24EC25F0000E89258A6F8B6BCC
:10323000000E8B238C6B070E8C238D6B020E8D235F
:103240008AC081F08BC082F08CC083F08DC084F086
:10325000010E856F000E17EC22F0816BFC0E826F61
:1032600083690F0E846F010E856F24EC25F07F0EAD
:10327000816F1C0E826F040E836F080E846F010E27
:10328000856F17EC22F0400E816F020E35D817ECD7
:1032900022F0816B826B836B846B010E856F030E52
:1032A00017EC22F0816B826B070E836F1A0E846F0E
:1032B000010E856F040E17EC22F0C00E816F030E15
:1032C0001BD817EC22F0816B826B040E836F020E09
:1032D000846F010E856F000E24EC25F01F0E0E0189
:1032E000466F6F6A6E38E832070BFBE1606A0F01C8
:1032F000306B788276821200826F836B846B010E52
:10330000856F020C010100056BE121EE09F07FD809
:10331000D8B4DF5C03E3030E0A6F096921EE09F0FC
:1033200071D8D8B4DF5C04E2FC0E0A6F010E096F9D
:1033300047512FE021EE09F011EE0DF05AD802E1CD
:10334000DF50E75C05E247510D27000E0E230DD03C
:1033500021EE0DF011EE09F04CD802E1DF50E75CF0
:1033600004E247510D5F000E0E5B4751116E126A69
:1033700009510D5D016E0A510E59026E03EC26F0E3
:103380000250800A136E1150015C1250800A1358CB
:1033900004E209C10DF10AC10EF121EE0DF037D89A
:1033A000D8B4DF5C03E3030E0E6F0D6921EE0DF060
:1033B00029D8D8B4DF5C04E2FC0E0E6F010E0D6F4D
:1033C0007DEC20F001C007F002C008F0A7EC17F078
:1033D0007DEC20F001C00FF002C010F048EF1EF0AD
:1033E000000E086A076AA7EC17F0106A0F6A48EF28
:1033F0001EF0E652DE52E550800A116EDD50800A62
:10340000115C1200DE52DD50800A840F020CDE5285
:10341000DD50800A7D0FFF0CE8CF01F05C500D0DF0
:103420000201000EF324D96E020EF420DA6E015070
:10343000E16EE26ADECFE6FFDECFE6FFDECFE6FF3B
:10344000DDCFE5FF5C5012EC0EF00150E16EE26A58
:10345000040EE126E26ADFCFE7FF5C500D0D050E9A
:10346000F324D96E020EF420DA6E0150E16EE26AA6
:10347000050EE126E26ADFCFE7FF5C500AEC0EF0B2
:103480000150E16EE26A060EE126E26ADFCFE7FF55
:103490005C5002EC0EF00150E16EE26A070EE1268C
:1034A000E26ADFCFE7FF5C5022EC0EF00150E16EE4
:1034B000E26A080EE126E26ADFCFE7FF5C501AEC11
:1034C0000EF00150E16EE26A090EE126E26ADFCFFA
:1034D000E7FF5C5032EC0EF00150E16EE26A0A0E3A
:1034E000E126E26ADFCFE7FF5C502AEC0EF00150E4
:1034F000E16EE26A0B0EE126E26ADFCFE7FF5C5085
:103500003AEC0EF00150E16EE26A0C0EE126E26A3E
:10351000DFCFE7FF5C2A0F0E5C165D065D160F0C11
:10352000AA51A91115E0A907D8A0AA070001AA511C
:10353000A9110EE1030E086E840E076E096A030ED0
:103540000B6E840E0A6E000E0D6A0C6A46EC1FF0BC
:10355000B66705D0B56703D08B9A8B981200B2512D
:10356000B1110EE1AF07D8A0B0070001B051AF1103
:1035700042E1ADC0B1F0AEC0B2F0B6C05FF03BD03A
:10358000B051AF110EE1B107D8A0B2070001B2519E
:10359000B11131E1ABC0AFF0ACC0B0F0B5C05FF07D
:1035A0002AD0ABC0AFF0ACC0B0F0B16BB26B23D0DF
:1035B0008B8A8B9812008B9A8B8812008B38010BA8
:1035C0000F6E8B38E832010B0F1805E1010E8BB836
:1035D000000E0F6E1AD8010E8BBA000E0F6E15D8A2
:1035E000010E8BB8000E0F6E0F3A8B500F18EF0BB9
:1035F0000F188B6E12005F50AFE0010ADCE0030A87
:10360000D7E0010AD8A41200D9D70F3A0F468B5041
:103610000F18DF0B0F188B6E1200646721D060C08B
:10362000D9FF61C0DAFFDF50656FD8906537D89059
:103630006537D8906535686F56D8D8906533662F52
:10364000FCD76551696F47D8656F050E666FD890D6
:103650006533662FFCD7655168136A6B6B6B2ED090
:1036600060C0D9FF61C0DAFFDF5046D86B6F3BD82E
:10367000D8906537662FFCD765516A6F676B2BD87A
:1036800002E0010E676F6739E8461F0B6A1320EEF0
:1036900002F06051D9266151DA22DF50696F1BD8E0
:1036A0002BD81C0B6A1317D8030B6A1320EE03F0F8
:1036B0006051D9266151DA22DF50686F62C0D9FFAC
:1036C00063C0DAFF68C0DEFF69C0DEFF6AC0DEFFEC
:1036D0006BC0DEFF120020EE01F06051D92661516F
:1036E000DA22DF50120060C0D9FF61C0DAFFDF507C
:1036F000656F050E666F050C656FD8906533D890C1
:103700006533D89065311200786714D074C079F0B1
:1037100075C07AF076C07BF077C07CF0040E01D0E3
:103720005AD8E82EFDD779514AD87439E846E00BCB
:10373000DF6E120074C079F075C07AF076C07BF04D
:1037400077C07CF0160E01D046D8E82EFDD779510F
:1037500036D874C079F075C07AF076C07BF077C047
:103760007CF0110E01D037D8E82EFDD7030E791763
:1037700074C07DF075C07EF076C07FF077C080F0B9
:103780000E0E05D0D89080337F337E337D33E82E04
:10379000F9D77D51E00B79110809DF6E20EE02F0B8
:1037A0007251D9267351DA2275C0DFFF20EE03F083
:1037B0007251D9267351DA2274C0DFFF120072C031
:1037C000D9FF73C0DAFFDF6E20EE01F07251D92607
:1037D0007351DA221200D8907C337B337A337933F9
:1037E0001200076614D003C008F004C009F005C039
:1037F0000AF006C00BF0040E01D05AD8E82EFDD70F
:1038000008504AD80338E846E00BDF6E120003C0C8
:1038100008F004C009F005C00AF006C00BF0160E4F
:1038200001D046D8E82EFDD7085036D803C008F09E
:1038300004C009F005C00AF006C00BF0110E01D05B
:1038400037D8E82EFDD7030E081603C00CF004C0CD
:103850000DF005C00EF006C00FF00E0E05D0D8908A
:103860000F320E320D320C32E82EF9D70C50E00B2D
:1038700008100809DF6E20EE02F00150D926025030
:10388000DA2204C0DFFF20EE03F00150D9260250F7
:10389000DA2203C0DFFF120001C0D9FF02C0DAFF45
:1038A000DF6E20EE01F00150D9260250DA2212001C
:1038B000D8900B320A3209320832120021EE50F051
:1038C000000EDE100001C86F240E52D800C1CDF0EA
:1038D00005C1CEF0010106510001CF6F02C1D0F049
:1038E0000DC1D1F001010E510001D26F19C1D3F009
:1038F00001011A510001D46F5BEC0BF075EC10F074
:1039000021EE50F0000EDE100001C86F280E30D8F6
:1039100048C1CDF0010149510001CE6F4AC1CFF03D
:1039200001014B510001D06FD16BD26BD36BD46BC3
:103930005BEC0BF075EC10F021EE50F0000EDE1099
:103940000001C86F2C0E14D823C1CDF024C1CEF0D5
:1039500025C1CFF026C1D0F01FC1D1F020C1D2F0D7
:1039600021C1D3F022C1D4F05BEC0BF075EF10F065
:10397000DE10C96F070EDE10CA6F020EDE10CB6FAD
:10398000080ECC6F080C1C341D34226E226605D044
:103990001A6A1B6A1C6A1D6A120020342134286EC0
:1039A000286605D01A6A1B6A1C6A1D6A1200285014
:1039B0007B0F22261DC028F02150281A800E2816C1
:1039C0001C8E208E216A236A246A256A266A070EC5
:1039D000276E1AA002D01E502BD832D81E361F36A2
:1039E00020362136272EF5D7110E276E1AA002D0C9
:1039F0001E501ED825D82632253224322332272EB7
:103A0000F5D723C001F024C002F025C003F026C082
:103A100004F022C005F028C006F0EAEC1DF004C056
:103A20001DF003C01CF002C01BF001C01AF0120010
:103A300023261F5024222050252221502622120006
:103A4000D8901D321C321B321A32D8901200E8CFA7
:103A500089F0800E6F6E948C948E02D0800E6F6E03
:103A60006E38E832070B040AF9E1800E726EE00E40
:103A70000E017D6F0ED0930E05D08F0E03D0830EF6
:103A800001D0810E0E01436FB80E446F050E456FD5
:103A90000AD000018951EFE0010AEFE0030AEFE0EC
:103AA000010AEFE0ECD7100E716F320E726F540EF8
:103AB000736F760E746F980E756FBA0E766FDC0E9C
:103AC000776FFE0E786F00011DD8000E24EC25F0F4
:103AD00019D824EC25F0816B826B836B846B010E0B
:103AE000856F000E17EC22F0010E0E01466F6F6A13
:103AF0006E38E832070BFBE1606A0F01306B7882A9
:103B000076821200816B826B836B846B010E856FF2
:103B1000010C21EE50F0000EDE100001C86F240EE3
:103B2000B8EC1CF000C1CDF005C1CEF0010106518A
:103B30000001CF6F02C1D0F00DC1D1F001010E51D3
:103B40000001D26F19C1D3F001011A510001D46FE5
:103B50003AD877EC0BF021EE50F0000EDE100001A9
:103B6000C86F280EB8EC1CF048C1CDF001014951D6
:103B70000001CE6F4AC1CFF001014B510001D06F5F
:103B8000D16BD26BD36BD46B1ED877EC0BF021EEDC
:103B900050F0000EDE100001C86F2C0EB8EC1CF0C7
:103BA00023C1CDF024C1CEF025C1CFF026C1D0F085
:103BB0001FC1D1F020C1D2F021C1D3F022C1D4F075
:103BC00002D877EF0BF0000E826FC80E816F010EE6
:103BD000836F010C055005E0045001100210031022
:103BE00007E1016A026A036A046A1200052A4AD8D8
:103BF000076A086A096AFE0E04140A6E0A50071062
:103C00000810091008E0F2D7052A012A000E022246
:103C10000322042237D8076A086A096A04500A6E28
:103C20000A5007100810091007E0EED70506D890D3
:103C3000013602360336043603AEF8D705B002D09B
:103C40007F0E0316D890053205C007F0086A096A8E
:103C50000A6A07C00AF0096A086A076A075001126F
:103C600008500212095003120A5004120650D8A438
:103C7000048E01C001F002C002F003C003F004C0D2
:103C800004F01200D89004320332023201321200E2
:103C900010500F1013E10C510B110BE0086A640E69
:103CA000076E096A0B6A0A6E000E0D6A0C6A46EC12
:103CB0001FF00FC00BF110C00CF112000FC00BF180
:103CC00010C00CF10FC001F010C002F0046A020E27
:103CD000036E55EC22F001C00FF002C010F000514D
:103CE000040AD8B412001050800A800F010ED8B414
:103CF0000F5C13E30F28076E000E1020086E096A90
:103D00000F5000080A6E1050D8A0E82A02080B6E67
:103D10000D6A0C6A010E46EF1FF010AE12000F5034
:103D20000108076E1050D8A0E82A0008086E000E9F
:103D3000096A0F240A6E020E10200B6E0D6A0C6ABF
:103D4000020E46EF1FF0E8CF39F0FF0E186E120E8C
:103D5000176EC4C019F0C5C01AF0C6C01BF0C7C0AA
:103D60001CF03950D96EDA6AC00EDE141D6EFF0EDB
:103D7000DE141E6EFF0EDE141F6E1F0EDE14206E8C
:103D80003950D96EDA6ADECF21F0DECF22F0DECFF5
:103D900023F0DECF24F0395054EC0BF0256E266A68
:103DA00074EC08F0376A386A0ED0FF0E186E1F0EDA
:103DB000176E395037244DEC0BF0196E1A6A74ECFB
:103DC00008F0374A382A395054EC0BF0346E356A13
:103DD0003850800A366E3450375C3550800A365879
:103DE000E4E3FE0E186EFE0E176E74EF08F0E8CFD7
:103DF00009F041D00950D96EDA6A0C0ED926DA6A78
:103E0000DF50016E0950D96EDA6A0B0ED926DA6AD4
:103E1000DF50026E0950D96EDA6A0A0ED926DA6AC4
:103E2000DF50036E0950D96EDA6A090ED926DA6AB4
:103E3000DF50046E0950D96EDA6A080ED926DA6AA4
:103E4000DF50056E09501BD8066E0950D96EDA6A2C
:103E5000060ED926DA6ADF50076E09504DEC0BF0DA
:103E60000724062405240424032402240124086EC4
:103E70000866000C010C095002D8BCE0000CD96E99
:103E8000DA6A070ED926DA6ADF501200E8CF0EF0A0
:103E90000D500001AA1902E10C50A91913E10E50AE
:103EA000B56310D00950B6630DD00850AC1902E1CB
:103EB0000750AB1907E10B50AE1902E10A50AD19DA
:103EC000D8B41200310E0C5C750E0D5804E3750E5B
:103ED0000D6E300E0C6E0CC0A9F00DC0AAF0E30EF2
:103EE000075C040E085804E3040E086EE20E076E29
:103EF000E30E0A5C040E0B5804E3040E0B6EE20E94
:103F00000A6E0EC0B5F009C0B6F007C0ABF008C02D
:103F1000ACF00AC0ADF00BC0AEF0ABC0AFF0ACC0BF
:103F2000B0F0B16BB26B1200E8CF13F01350D96E42
:103F3000DA6A0001DECFC8F0DECFC9F0DECFCAF00A
:103F4000DECFCBF0135054EC0BF0CC6F13504DEC94
:103F50000BF0CD6F1350D96EDA6A060ED926DA6AE5
:103F6000DF50CE6F13503FEC1FF0CF6F1350D96E60
:103F7000DA6A080ED926DA6ADF50D06F1350D96E8C
:103F8000DA6A090ED926DA6ADF50D16F1350D96E7A
:103F9000DA6A0A0ED926DA6ADF50D26F1350D96E68
:103FA000DA6A0B0ED926DA6ADF50D36F1350D96E56
:103FB000DA6A0C0ED926DA6ADF50D46F5BEC0BF0AC
:103FC00075EF10F00D340E34146E146605D00B6AC4
:103FD0000C6A0D6A0E6A12000BC00FF00CC010F0D4
:103FE0000DC011F00EC012F0200E05D0D890123284
:103FF000113210320F32E82EF9D70F50136E0D8E9A
:104000000E6A960E145E14AE0CD01450800A970FF0
:10401000DEE3D8900E320D320C320B32143EF9D75B
:104020000CD01F0E146407D0D2D7D8900B360C36A4
:104030000D360E3614061466F8D7135008E00E1E1F
:104040000D1E0C1E0B6C000E0C220D220E220BC03E
:104050000BF00CC00CF00DC00DF00EC00EF01200F5
:10406000E8CF79F07851AA1902E17751A91913E143
:104070007951B56310D07451B6630DD07351AC193A
:1040800002E17251AB1907E17651AE1902E17551A7
:10409000AD19D8B41200310E775D750E785904E36E
:1040A000750E786F300E776F77C0A9F078C0AAF0E0
:1040B000E30E725D040E735904E3040E736FE20E97
:1040C000726FE30E755D040E765904E3040E766F8D
:1040D000E20E756F79C0B5F074C0B6F072C0ABF087
:1040E00073C0ACF075C0ADF076C0AEF0ABC0AFF051
:1040F000ACC0B0F0B16BB26B120080AE03D0010166
:10410000028102D00101029180AC02D0028301D071
:10411000029302AD0FD021EE0DF0DECF03F0DDCF24
:1041200004F0031E041E034A042A03C005F004C061
:1041300006F004D00DC105F00EC106F002A522D094
:1041400002A70CD00650800A800F010ED8B4055C7F
:10415000D8B080AE0CD0016A026A12000650800A04
:10416000800F010ED8B4055C02E380AEF4D702A93B
:1041700005D006AE07D080BCEED704D006AE02D084
:1041800080ACE9D70DC101F00EC102F01200FF0EA4
:10419000186E400E176E74EC08F0700ED3129B8CE4
:1041A000800E6F6EC00E946E550E8B6E0AEC27F06B
:1041B00002D0800E6F6E6E38E832070B040AF9E108
:1041C000810E0E01436FB80E446F050E456F726A83
:1041D0007D6B716B726B736B746B756B766B776BDE
:1041E000786BE069E169E269E369F86BF96BFA6B96
:1041F000FB6B01D06F6A6E38E832070BFBE1400EB3
:10420000606E0F01306FAA0E8B6EFE0E186E5C0E84
:10421000176E74EC08F001EF00F0120021EE50F080
:10422000000EDE100001C86F440EB8EC1CF0026AEC
:10423000380E016E70EC26F00001CD6F026A390E67
:10424000016E70EC26F00001CE6F026A3A0E016E2C
:1042500070EC26F00001CF6F026A3B0E016E70EC2D
:1042600026F00001D06F026A3C0E016E70EC26F061
:104270000001D16F026A3D0E016E70EC26F0000164
:10428000D26F026A3E0E016E70EC26F00001D36F11
:10429000026A3F0E016E70EC26F00001D46F5BECF9
:1042A0000BF075EF10F021EE50F0000EDE10000163
:1042B000C86F380EB8EC1CF0026A400E016E70EC4C
:1042C00026F00001CD6F026A410E016E70EC26F0FF
:1042D0000001CE6F026A420E016E70EC26F0000102
:1042E000CF6F026A430E016E70EC26F00001D06FB2
:1042F000026A440E016E70EC26F00001D16F026A72
:10430000450E016E70EC26F00001D26F026A460E77
:10431000016E70EC26F00001D36F026A470E016E49
:1043200070EC26F00001D46F5BEC0BF075EF10F031
:1043300001014D670CD0000E086A076AA7EC17F060
:10434000086A320E076E096A0B6A640E0CD04C675D
:1043500017D0000E086A076AA7EC17F0086A640E07
:10436000076E096A0B6A0A6E0D6A0C6A030E46EF45
:104370001FF082EF19F012001200120063EF0FF02D
:104380000151F7E0010AD8B41200030AF4E0010A6F
:10439000D8B41200070AF0E0010AD8B41200030AE8
:1043A000ECE0010AD8B412000F0AE8E0010A12009A
:1043B000B1EC26F001C02FF002C030F030AE02D0D8
:1043C0002F6A306ABBEC26F001C02DF002C02EF03F
:1043D0002EAE02D02F6A306A1E6A1F6A880E206EC7
:1043E000400E216E2D502F5C156E2E503058166EDB
:1043F00043EC25F018C01DF017C01CF016C01BF0D0
:1044000015C01AF0C3EC1CF01DC00EF01CC00DF05E
:104410001BC00CF01AC00BF0E2EC1FF00BC02BF02D
:104420000CC02CF02BC029F02CC02AF01200E8CFD1
:1044300086F020D00E0E0001886FE00E18D00E0E10
:104440000001886FE40E13D00E0E0001886FE80E95
:104450000ED00E0E0001886FEC0E09D00E0E00017A
:10446000886FF00E04D00E0E0001886FF40E00016C
:10447000876F0BD08651DEE0010AE1E0030AE4E039
:10448000010AE7E0070AEAE0EED787C072F088C0C9
:1044900073F081C074F082C075F083C076F084C080
:1044A00077F085C078F084EF1BF0066A04AE06D082
:1044B000036C041ED8B0042A010E066E02AE06D0AC
:1044C000016C021ED8B0022A010E061A076A086A99
:1044D000045003101BE0010E056E04D0D890033683
:1044E0000436052A04AEFAD7D890073608360350AA
:1044F000015C0450025805E30350015E0450025A67
:104500000780D89004320332052EEED7065004E01F
:10451000076C081ED8B0082A07C001F008C002F0D6
:1045200012007A6B7B6B7C6B7D6B79517611771106
:10453000781129E0010E7E6F06D0D8907637773754
:10454000783779377E2B79AFF8D7D8907A377B37A1
:104550007C377D377651725D775173597851745934
:104560007951755909E37651725F7751735B7851D0
:10457000745B7951755B7A81D8907933783377336E
:1045800076337E2FE2D77AC072F07BC073F07CC0A6
:1045900074F07DC075F01200E8CF3CF03C50D96E4D
:1045A000DA6AC00EDE14386EFF0EDE14396EFF0EAE
:1045B000DE143A6EFF0EDE143B6E0FD03C5062EC00
:1045C0000BF000C1CDF05BEC0BF075EC10F0FE0EC3
:1045D000186EF00E176E74EF08F038C034F039C062
:1045E00035F03AC036F03BC037F03750020AD8A455
:1045F000120008D03550140AD8A412003450D8A4A0
:104600001200DCD73650070AD8A41200F3D7096A83
:104610000A6A0B6A0C6A085005100610071029E098
:10462000010E0D6E06D0D8900536063607360836D0
:104630000D2A08AEF8D7D89009360A360B360C3654
:104640000550015C065002580750035808500458A2
:1046500009E30550015E0650025A0750035A0850FC
:10466000045A0980D89008320732063205320D2EDE
:10467000E2D709C001F00AC002F00BC003F00CC081
:1046800004F01200700ED3129B8C9496829689ECE3
:104690001DF0030E27EC1DF0030EEDEC18F05C6B23
:1046A0005D6BF00E5B6FF19E5C6B5D6B949694841A
:1046B000928E928CA7EC26F058EC26F017EC26F0A0
:1046C00088EC26F09DEC26F093EC26F003EC27F026
:1046D0004CEC26F0000E0001776B766B48EC16F080
:1046E000D08EF28CF28E27EF26F086518311841142
:1046F000851123E0010E876F06D0D8908337843769
:1047000085378637872B86AFF8D783517F5D8451F5
:104710008059855181598651825908E383517F5FC1
:104720008451805B8551815B8651825BD890863352
:10473000853384338333872FE8D77FC07FF080C0F1
:1047400080F081C081F082C082F01200E8CF14F0C6
:10475000156A14501524D96EDA6A050ED926DA6A5C
:104760001F0EDF6411D0145015244DEC0BF0136EA6
:104770007F0E135C09E214D8145015244DEC0BF095
:10478000036E60EC25F004D00BD8036A60EC25F0D2
:1047900007EC27F0152A070E1564DBD753EF21F03D
:1047A000400E1524016E026A000E0222000C155004
:1047B00012101310141023E0010E166E06D0D890BC
:1047C0001236133614361536162A15AEF8D712508F
:1047D0000E5C13500F58145010581550115808E320
:1047E00012500E5E13500F5A1450105A1550115A91
:1047F000D8901532143213321232162EE8D70EC06A
:104800000EF00FC00FF010C010F011C011F0120028
:10481000050EC26EC282C2B2FED7770E1E6EBE0EEB
:104820001F6EBF0E206E3F0E216EC3CF15F0C4CF9A
:1048300016F0DAEC25F018C01DF017C01CF016C0F9
:104840001BF015C01AF0C3EC1CF01DC00EF01CC00C
:104850000DF01BC00CF01AC00BF0E2EC1FF00BC007
:1048600029F00CC02AF01200010EC26EC282C2B240
:10487000FED7770E1E6EBE0E1F6EBF0E206E3F0E51
:10488000216EC3CF15F0C4CF16F0DAEC25F018C0B6
:104890001DF017C01CF016C01BF015C01AF0C3ECB9
:1048A0001CF01DC00EF01CC00DF01BC00CF01AC097
:1048B0000BF0E2EC1FF00BC029F00CC02AF0120044
:1048C000B46705D0026A010E016EC5EC26F0A5C0E2
:1048D00001F0A6C002F0A7C003F0A8C004F06D0E5E
:1048E000056E4E0E066EC60E076E410E086EDAECB1
:1048F00024F0390E01240001A56F300E0220A66FAE
:10490000000E0320A76F000E0420A86FA7510D6EA4
:104910007F0EA8150E6E120021EE50F0000EDE1074
:104920000001C86F300EB8EC1CF0010ECD6F050E03
:10493000CE6F7CEC26F00150CF6FD06B030E026E71
:10494000FD0E016E70EC26F00001D16F030E026EB9
:10495000FE0E016E70EC26F00001D26FD36BD46BAB
:104960005BEC0BF075EF10F004AE09D0016C021E89
:10497000D8B0022A031ED8B0032A800E045608AE0F
:1049800009D0056C061ED8B0062A071ED8B0072A23
:10499000800E0856800E041A081A0550015C065055
:1049A0000258075003580850045802E2D8901200E9
:1049B000D8801200096A0A6A0B6A0C6A01A008D042
:1049C0000550092606500A2207500B2208500C22D7
:1049D000D8900536063607360836D89004320332AA
:1049E000023201320450011002100310E7E109C045
:1049F00001F00AC002F00BC003F00CC004F012007A
:104A00000F6A0EAE0AD00E1E0D1E0C1E0B6C000E91
:104A10000C220D220E22010E0F6E0BC001F00CC0F5
:104A200002F00DC003F00EC004F0960E056E0FC02C
:104A300006F0EAEC1DF004C00EF003C00DF002C059
:104A40000CF001C00BF01200E8CF86F0866705D0AD
:104A50000E0E0001886FF80E04D00E0E0001886F54
:104A6000FC0E0001876F87C072F088C073F081C0B0
:104A700074F082C075F083C076F084C077F085C092
:104A800078F084EF1BF0196A16AE05D0156C161E6F
:104A9000D8B0162A192A15C001F016C002F0036A10
:104AA000046A960E056E19C006F0EAEC1DF004C00B
:104AB00018F003C017F002C016F001C015F0120084
:104AC0000250030B756E01C074FF03C073FF7F9E1D
:104AD0007F9C7F84000EF2BE010E046EF29E550E86
:104AE0007E6EAA0E7E6E7F827FB2FED704B002D0A9
:104AF000F29E01D0F28E7F94120002EE00F0D00EF2
:104B0000EE6AE806FDE101EE00F0540EEE6AE806FA
:104B1000FDE100EEA5F0230EEE6AE806FDE15F6A16
:104B20005E6A5D6A5C6A000152EF18F00150030290
:104B3000F3CF05F0F4CF06F00150040208D802507C
:104B4000030205D805C001F006C002F01200F3CF41
:104B5000F4FFF36AF3500526F45006221200F3CF57
:104B600070F0F4CF71F077A201D001D005D0500ED3
:104B700001014D6FE5EC0CF071C0F4FF70C0F3FF64
:104B80006FC0DAFF6EC0D9FF1100E8CF73F00CD010
:104B9000170ECFEC26F0170ECFEC26F0170ECFEC49
:104BA00026F0170ECFEC26F0000173077329D8B456
:104BB0001200EED715C001F016C002F0036A046AB5
:104BC000960E056E000E066AEAEC1DF004C018F0A1
:104BD00003C017F002C016F001C015F0120073AF49
:104BE0000DD072C074F073C075F0741F751F744BD4
:104BF000752B74C072F075C073F0120072C072F041
:104C000073C073F0120002AE0DD001C003F002C0F9
:104C100004F0031E041E034A042A03C001F004C06A
:104C200002F0120001C001F002C002F01200949ADA
:104C300094988B8A8B980001736BC80E726F746B9B
:104C4000766B756F000E786B776B30EF20F001019B
:104C50000005D8A41200949682960A0EC5EC25F0A1
:104C60008286010EC5EF25F0746B80BA748182B024
:104C7000748382B27485742B74C072F0736B1200EB
:104C80007351030B756E72C074FF7F9C7F9E7F8093
:104C900000F000F073501200FFEC26F09392939412
:104CA000939693984C0EBB6E996A800EBC6E800CE6
:104CB000900EA66E240EBA6E938C939E080EB96E5B
:104CC0008A0E7B6E7C6A120008D00001B70E0CECD5
:104CD0001AF00001B70E5AEC04F05D66F6D7120028
:104CE0000250030B756E01C074FF7F9C7F9E7F8016
:104CF00000F000F073501200036A80BA038082B0A3
:104D0000038282B20384032A03C001F0026A120004
:104D10009280010EC26E300EC16EA50EC06E0F01E4
:104D20005D81C282A50C9284010EC26E300EC16EEE
:104D3000A50EC06E5D85C282A50C9284010EC26E66
:104D4000300EC16EA50EC06E5D87C282A50C800EAE
:104D5000D56EE00ED76ECF0ED66EF294F28AF19435
:104D6000CF0C0D0EC26EC282C2B2FED7C3CF01F00D
:104D7000C4CF02F01200090EC26EC282C2B2FED7C8
:104D8000C3CF01F0C4CF02F01200000101C0A5F0B2
:104D900002C0A6F0A76BA86B010EB46F010CE8CFA0
:104DA00072F0000172077229D8B41200FAD7E8CF66
:104DB00072F0A4A8FED772C079FF120008EC24F0AC
:104DC00029C02BF02AC02CF01200E8CF01F0010618
:104DD0000128D8B41200FBD7E8CF01F0A4A8FED771
:104DE00001C079FF1200E8CF72F0000172513F0B51
:104DF00012000005D8A41200949682861200070EB5
:104E0000CA6ECB681200928A9480948212007FA2AC
:104E10001200FDD794968296120012001200120022
:10FD7000010000000A00000064000000E803000029
:10FD800010270000A086010040420F0080969800D6
:10FD900000E1F50500CA9A3B0100000010000000D8
:10FDA0000001000000100000000001000000100031
:10FDB0000000000100000010534435343043202D72
:10FDC0002025732046572D25642E25642048572D65
:10FDD00025642E256420424C2D25642E25640D0AB1
:10FDE00000756D7077723D2025642063706F7765B4
:10FDF000723D25642073703D25640D0A004C4D5FF3
:10FE00004150495F4346475F4252414B455F434F34
:10FE10004153540D0A004C4D5F4150495F434647E2
:10FE20005F4C494D49545F4D4F44450D0A004C4DC0
:10FE30005F4150495F4346475F504F545F545552AE
:10FE40004E530D0A004C4D5F4150495F4346475F9A
:10FE50004C494D49545F5245560D0A000D0A5F5FEB
:10FE60005F6D6B7374722820424F4F544C4F414466
:10FE700029200053443534305F4346475F4C494D99
:10FE800049545F4657440D0A004C4D5F4150495F4D
:10FE90004346475F4D41585F564F55540D0A000D7C
:10FEA0000A4C4D5F4150495F5550445F5245515592
:10FEB00045535420004C4D5F4150495F4346475FD6
:10FEC0005245565F4657440D0A000D0A53443534D7
:10FED0003043205265626F6F74696E670D0A00309F
:10FEE00031323334353637383961626364656600E0
:10FEF0004C4D5F4150495F535441545553200D0AB6
:10FF00000025782025782020257820202578200DB0
:10FF10000A00256C7520256C7820256C782020251A
:10FF20007820000D0A4C4D5F4150495F5550447890
:10FF300020000D0A676F746F426F6F7428292000CC
:10FF40000D0A696E20676F746F426F6F74004465AD
:10FF5000765365724E6F20697320004465764E615A
:10FF60006D6520697320004A616E20303220323086
:10FF7000313700535953524553554D45200049449C
:10FF8000206368616E6765200044455651554552AF
:10FF9000592000256C78206E6F6E652000466972CE
:10FFA0006D776172652000426C696E6B204C454430
:10FFB000004E4F4E20535953200053595348414C43
:10FFC0005420005359535253542000286E756C6CC2
:10FFD0002900494354524C200056434F4D502000B5
:10FFE0005053544154200053594E43200053504421
:10FFF00020004346472000504F5320002E21000090
:00000001FF
